:02000000F629DF
:1000080003088D00820700000000000000000000C7
:1000180000000000000000000000000000000000D8
:1000280000000000000000000000000000000000C8
:100038000800C60A08304602031D2428C601C60A5D
:10004800460882072E283B284828552862286F280A
:100058007C288928FF304602031D3A28C60A033047
:100068004602031D3A28C601013086061D28FF30C6
:100078004602031D4728C60A08304602031D4728C2
:10008800C601023086061D28FF304602031D54288B
:10009800C60A06304602031D5428C60104308606E7
:1000A8001D28FF304602031D6128C60A0B30460290
:1000B800031D6128C601083086061D28FF30460248
:1000C800031D6E28C60A0C304602031D6E28C601A1
:1000D800103086061D28FF304602031D7B28C60AFD
:1000E80004304602031D7B28C601203086061D28E1
:1000F800FF304602031D8828C70A17304702031D30
:100108008828C701403086061D28FF304602031D97
:100118009528C70A09304702031D9528C701803072
:1001280086061D28000000001108062000000000B7
:10013800120806208F0B962808000E34113411344B
:100148000A340434043411341B3415341134113492
:100158000E341F34013401340234023404340434BC
:100168000E3404340C340434043404348D01640033
:100178008E30620007308E008518CD28051DC028F6
:10018800851103108D0C851CC72885158E0BC0287A
:10019800D7280519C028051003148D0C051DD22871
:1001A80005148E0BC0288518DC28051DD728E228E1
:1001B8000519D728131403148D0C08001310031005
:1001C8008D0C080007308C00DE2904308C00DE29F5
:1001D8007E3430346D34793433345B345F34703486
:1001E8007F34733477341F344E343D344F344734BE
:1001F8008612000006088D00861608000611000009
:100208000D08860006150800003066002D308600AF
:1002180006114708860000000615061008008D0123
:1002280064008C30620008308E0085182629051D70
:100238001929851103108D0C851C202985158E0B15
:100248001929080005191929051003148D0C051D15
:100258002B2905148E0B1929080010308F008610E1
:1002680086110E30062086148615113006208F0B55
:100278003329080086140611000048088600061570
:100288000000061100004908860006150000061146
:1002980000004A0886000615000086100800132191
:1002A8000D08860006288617061F58298613080099
:1002B8000030660013210D0886000628FF3066000E
:1002C80006088D00B0210628C90DC90DCA0DC90D33
:1002D800CA0DC90DCA0D0F30C90508000430C80081
:1002E800CA014808C900682149088C0006160000A0
:1002F800C70108213E21FF30660057214710FC2026
:10030800FE300D0203198C294714CA01CB010800DD
:10031800FC200D08CA000D08C800FC200D08CB0001
:100328000D08C9008C038C080319AF292030C807B1
:10033800031CA229C90A031CA229CA0AC908031D49
:10034800A92920304802031C7A292030C802031C3E
:100358009A29C9039A29080064008C306200083081
:100368008E00851CB529051DB52903108D0C0318B1
:10037800C62905100519BE290514051DC1298E0BAE
:10038800B529CE2985118518C7298515851CCA293F
:100398008E0BB529851CCE29051DCE2908009B305A
:1003A8008C0064008C30620000008C0BD829080097
:1003B80010308F000C3006200F3006208F0BDE29FE
:1003C800080008308F00DE290D308F00DE298610E6
:1003D80086111108062086148615120806208F0B30
:1003E800EB290800063065003430660019308500B6
:1003F8000A30860064008C3062000516061DC02A8B
:10040800861E082A061A0C2A0519851CFA2AFE29AE
:100418000508063912060319FE2905120508920077
:10042800063092053121051D1B2A31211C2ADC21A9
:10043800851C202A3121212ADC21E821DC21FE2902
:10044800C801CA0113210D08C9006821C701082184
:100458003E21FF3066005721FC2088300D02031929
:10046800392A8D01B0210616062808308C00FC2098
:10047800B0218C0B392A0616062813210D08C8004E
:1004880013210D08C90072214A088D00B0214B08BC
:100498008D00B021471C532A061647100628FC2059
:1004A8000D088C00B0218C0AFC20B0218C0B582A36
:1004B8000616062813210D08C80013210D08C900C7
:1004C80072214A088D00B0214B088D00B021471CCD
:1004D800702A061647100628FC200D088C00B0214B
:1004E8008C0A0C08CA07031C7A2ACB0A1D308C0018
:1004F800FC20B021CA03031C842ACB030318652AF5
:100508008C0B7C2A0512E5210619FE29DC21061927
:100518000D11061D0D15DC2106198D10061D8D14F3
:100528000D199B2A051D9D2A851112119D2A8515D5
:1005380012158D18A42A851CA62A05109210A62A21
:1005480005149214D321E8210C2A1321A1300D029D
:100558000319242AA2300D020319412A12300D0270
:1005680003195C2910300D020319622914300D0299
:10057800031953295721A92A861EC52A061A862A2D
:10058800FE298D010512061EDA2AE5210619FE2923
:10059800DC210619D42A05101310061DD12AD62AE3
:1005A800851113140619D62A0730DB2A08308E0065
:1005B800E5210619FE29DC21061D0310061903147E
:1005C8008D0C8E0BDF2ADC210619FE29061EF72A60
:1005D8008D0C08308E00131CF32AC621F42ABD2185
:1005E800DC213121F82AB021E821FE290512861ADA
:1005F800422B061E2C2B3121051D042B3121052BE6
:10060800DC21E821BA208D0C07308E00312103103F
:100618008D0C0318112B3121122BDC218E0B0B2B87
:100628003121E8210619162B061D182B131C1E2B29
:1006380005108A1B85118518232B051D1F2B0514F2
:100648008515851C252B051D252BE821DC21FE2978
:10065800132108308E00312103108D0C0318382B1C
:1006680031218E0B302B3B2BDC218E0B302B312193
:10067800E821D321D321D321D321FE2913218D1B96
:10068800F22B0D0890008C0013210D088F00132108
:100698000D08910013210D0892000C1BC52B133077
:1006A800840013210D088000840A8C0B552B13300D
:1006B80084000F088D0008308E000D088F0064003C
:1006C8008C3062000310800D031C6C2BEB216D2B0A
:1006D80096208E0B612B840A900B5F2BD321FE2969
:1006E800C6000830C600051064000B308100051CE8
:1006F8007B2B4508C5000000C50B7F2BC5000030CB
:10070800C60C031C8D2B65000130C50B882B6500BA
:10071800942B65000130902B912BC50B8E2B650017
:10072800C60B7D2B4508C5000000C50B982B64003F
:1007380008000830C600051064000B308100051C55
:10074800A32B4508C500003065000130C50BA92B57
:100758006500AE2BAF2BB02BC5010518B12BC50A10
:1007680045084502051CB32BC60CC60BB02B051853
:10077800BB2B64000800003066000730C600C601C5
:1007880086016400051DFE29851CFE290619C52B56
:100798008C3062003F308C059005133084000F08C0
:1007A8008D008F0C962008308E0064008C3062001B
:1007B8000D088F0006190310061D0314800D9620DE
:1007C8008E0BDC2B840A900BD72B13308400000887
:1007D8008D00B021840A8C0BEB2BFE290D1BF92B05
:1007E8000608C1398D00B021FE290D08C1393438F9
:0807F80066000A308600FE29AC
:1042000000000000000000000000000000000000AE
:10421000000000000000000000000000000000009E
:10422000000000000000000000000000000000008E
:10423000000000000000000000000000000000007E
:10424000000000000000000000000000000000006E
:10425000000000000000000000000000000000005E
:10426000000000000000000000000000000000004E
:10427000000000000000000000000000000000003E
:084000007F007F007F007F00BC
:02400E00FD3F74
:02FFFE0084007D
:00000001FF
